:1000000000308A00BA2C00003E308400000803193A
:1000100018280130A100A001A00B0C28A10B0B286F
:100020002730A000A00B122800000000800B092838
:100030000034AE0A0319AF0A2E08603C031D2A28BB
:100040002F08EA3C031D2A28B00A3008A03C031DF3
:100050002A280510003403306600B501861C3228BA
:1000600019202E288618362819203228B401340881
:10007000073C031C482886183B283E28061C4128BC
:100080003514861C41284428350CB50CB40A372891
:10009000B4013408013C031C552886184D2850280B
:1000A000861C50285328B40A4928013066003508B8
:1000B000A10000340030660086101730A000A00BAD
:1000C0005F28000006100230A000A00B6528000089
:1000D000861402306600B601B5013508073C031CE2
:1000E000842886187128742834080139003A0319C5
:1000F0007C280614B60A7D280610340CB40C861C25
:100100007F288228B50A6D28861884288728360813
:100110000139003A031D8E2806148F280610861C0C
:100120008F28922886189228952806140330660096
:100130008610061899289C28061C9C289F280130A8
:1001400066000034ED30B4005A202B202908B4009A
:100150005A2000343908BD0006122830BE000420A1
:10016000BC013A083C020318ED283D08B900861589
:10017000BB013B08043C031CD32839080139003A71
:100180000319C4280615C52806110430A000A00BC9
:10019000C72886110430A000A00BCC288615390C86
:1001A000B90CBB0AB9283230BE0004200615BB01C9
:1001B0003B08043C031CE8280430A000A00BDE2808
:1001C00086110430A000A00BE3288615BB0AD828AE
:1001D0002330BE000420BC0AB128B001AF013008B2
:1001E000AE00061600346430BE00042001308500E5
:1001F000083086006430BE000420B001AF01300832
:10020000AE0000340030AC180130013C031D32292F
:10021000AD08031D15293408AD00B403340EA80041
:100220000310A80DE030A8053229280883169B008A
:100230009A011C1583120B08A0008B1355308316EE
:100240009D00AA309D009C14831283169C1C2A29B1
:10025000831225291C11831220088B001430BE0044
:100260000420AD010030AC180130003A031D85298F
:1002700001303402B500B600360EA8000310A80DF8
:10028000E030A805280883169B009C131C141A084C
:100290008312B7001430BE00042037080F39B800AD
:1002A000B70E0F30B705370B56295829003059299A
:1002B0000130B9003808083C03185F296129003073
:1002C000622901303905003A03196A290C30B70058
:1002D0000630B807A80A27083702031D74290D3015
:1002E000B9000130BA00AA20B708031979293708E4
:1002F000A7003708B9003808BA00AA206430BE0049
:100300000420B708031D4229A80100343208A000C8
:10031000F03020020319852A143020020319A82A7C
:10032000123020020319AA2A593020020319AA2ADE
:10033000583020020319AD2A773020020319BC2A55
:100340001C3020020319C02A323020020319C32AAC
:10035000213020020319C82A233020020319CD2A94
:10036000243020020319D02A2B3020020319D52A69
:10037000343020020319DA2A333020020319DD2A2F
:10038000433020020319E22A3B3020020319E72AF6
:10039000423020020319EA2A4B3020020319EF2AC7
:1003A0003A3020020319F42A313020020319F72AC7
:1003B000443020020319FC2A4D3020020319012B7E
:1003C000153020020319042B2D3020020319072BAE
:1003D0001B30200203190C2B2C3020020319112B87
:1003E0003C3020020319142B2A3020020319192B48
:1003F0001D30200203191E2B223020020319212B4D
:10040000353020020319262B1A30200203192B2B1A
:10041000163020020319302B1E30200203193B2B0B
:10042000263020020319462B253020020319512BB8
:100430002E3020020319592B363020020319642B69
:100440003D30200203196C2B3E3020020319772B1C
:100450004630200203197F2B4530200203198A2BD6
:10046000293020020319952B493020020319982BBB
:10047000413020020319A32B4A3020020319AE2B6E
:100480004C3020020319B92B523020020319C42B1F
:100490004E3020020319CF2B663020020319D72BD0
:1004A000E03020020319DF2B6B3020020319122CDD
:1004B000743020020319152CE13020020319182C86
:1004C0005A3020020319212C063020020319242C53
:1004D0000430200203192B2C7630200203192E2C15
:1004E0000C3020020319332C033020020319382C5E
:1004F0000B30200203193C2C833020020319402CBE
:100500000A3020020319442C482C2B202108B30068
:10051000A5013308123C031D8E2A902A0030912A2F
:100520000130B4003308593C031D972A992A003042
:100530009A2A01303404003A0319A22A2C100330FD
:10054000A905A2203308143C031DA72AAC10482C8F
:10055000AC14482C2C14A501482C0430A906A22068
:1005600000302C180130013A003A0319B82ABA2A8F
:100570002C10BB2A2C14482C0230A906A220482C8F
:100580000230A500482C0230A5000230A600482CFD
:100590000230A5000330A600482C0330A500482CEB
:1005A0000330A5000230A600482C0330A50003301C
:1005B000A600482C0430A500482C0430A5000230C9
:1005C000A600482C0430A5000330A600482C0530B6
:1005D000A500482C0530A5000230A600482C0530A7
:1005E000A5000330A600482C0630A500482C063094
:1005F000A5000230A600482C0630A5000330A60056
:10060000482C0730A500482C0130A500482C0730A5
:10061000A5000230A600482C0730A5000330A60034
:10062000482C0830A500482C0830A5000230A60050
:10063000482C0830A5000330A600482C0930A5003E
:10064000482C0930A5000230A600482C0930A5002E
:100650000330A600482C0130A5000230A600482C2B
:100660000130A5000330A6002C1C3A2B0C30A5004D
:100670000230A600482C0230A5000430A6002C1C35
:10068000452B0C30A5001230A600482C0330A500E5
:100690000430A6002C1C502B0C30A5000930A600FD
:1006A000482C0430A5000430A6002C1C582BA501B2
:1006B000482C0530A5000430A6002C1C632B0C3000
:1006C000A5000A30A600482C0630A5000430A6007C
:1006D0002C1C6B2BA501482C0730A5000430A6006C
:1006E0002C1C762B0C30A5000830A600482C0830B6
:1006F000A5000430A6002C1C7E2BA501482C093037
:10070000A5000430A6002C1C892B0C30A5000B3052
:10071000A600482C0A30A5000230A6002C1C942B01
:100720000C30A5000C30A600482C0A30A500482C3F
:100730000C30A5000430A6002C1CA22B0C30A50008
:100740000E30A600482C0C30A5000530A6002C1C4D
:10075000AD2B0C30A5000D30A600482C0C30A500A8
:100760000730A6002C1CB82B0C30A5000130A600C9
:10077000482C0C30A5000F30A6002C1CC32B0C30CD
:10078000A5001030A600482C0C30A5000330A600B0
:100790002C1CCE2B0C30A5001130A600482C0C30A0
:1007A000A5000630A6002C1CD62BA501482C0E3027
:1007B000B9000130BA00AA200F30A500482C2B2028
:1007C0002108B3006B3C031DEA2B0E30A5002B2043
:1007D0002B202B203308743C031DF32B0D30A50078
:1007E0002B202B202B203308123C031DFF2BB301A1
:1007F0003308073C031CFF2B2B20B30AF82B3308CC
:10080000713C031D052C0F30A5003308753C031DFA
:100810000B2C8515F3203308723C031D112C061791
:10082000F320482C0E30A500482C0D30A500482C94
:10083000B3013308063C031C202C2B20B30A192CCF
:10084000482C8616F320482C8514F3200617F32035
:100850008616F320482C0515F320482C8617F32024
:100860000515F320482C8514F3208616F320482C18
:100870000130B4000221482C0230B4000221482C7F
:100880000330B4000221482C0430B4000221482C6B
:100890002C1C542C2508093C031C502C0430A607A2
:1008A000250B542C0130A60225080C3C031C592CA6
:1008B0005B2C00305C2C0130B400A5080319612CBE
:1008C000632C0030642C01303405003A0319B42C39
:1008D00027082502031D712C0D30B9000130BA0024
:1008E000AA202508A700AD080319B42C2508AA00E2
:1008F0002608AB002B080F3C0318822C0630AB02F5
:100900000130AA002A0EA000F030A00520082B0715
:10091000AA00280883169B0083122A0883169A00CF
:100920001C1583120B08A0008B13553083169D00F5
:10093000AA309D009C14831283169C1CA12C831248
:100940009C2C1C11831220088B001430BE00042044
:100950002D0EA0000310A00DE030A0052008FF3EE2
:1009600028020318B42CA80A25080C3C0318B92C3B
:10097000A701E52C840107309F00A9012C10AC10C1
:10098000B001AF013008AE000330660010306500E2
:1009900083168113C8308312BE0004200130850005
:1009A00008308600061686108613051186128510FB
:1009B00085110613AD01A801A5010130A6002B2069
:1009C0002108B1003108B2008629A5080319ED2CD1
:0E09D0002508B9002608BA00AA20DC2C630016
:02400E00A13FD0
:1042000000000000000000000000000000000000AE
:10421000000000000000000000000000000000009E
:10422000000000000000000000000000000000008E
:10423000000000000000000000000000000000007E
:10424000000000000000000000000000000000006E
:10425000000000000000000000000000000000005E
:10426000000000000000000000000000000000004E
:10427000000000000000000000000000000000003E
:10428000000000000000000000000000000000002E
:10429000000000000000000000000000000000001E
:1042A000000000000000000000000000000000000E
:1042B00000000000000000000000000000000000FE
:0842C0000000000000000000F6
:00000001FF
